:0400000019EF18F0EC
:08000800056ED8CF06F0E0CF31
:1000100007F00001E9CF0DF0EACF08F0E1CF09F0D9
:10002000E2CF0AF0D9CF0BF0DACF0CF0F3CF14F017
:10003000F4CF15F0FACF16F000C00FF001C010F0A9
:1000400002C011F003C012F004C013F09DAA2CEFFF
:1000500000F09EBA52EF0AF00FC000F010C001F09D
:1000600011C002F012C003F013C004F00DC0E9FF8C
:1000700008C0EAFF088E09C0E1FF0AC0E2FF0BC01A
:10008000D9FF0CC0DAFF14C0F3FF15C0F4FF16C08F
:10009000FAFF055007C0E0FF06C0D8FF1000F2CFFE
:1000A0000EF0F29EF76AB80FF66E000EF722090006
:1000B000F5500EBEF28E120021303034302C253037
:1000C000364C5800F2CF0EF0F29EF76ADE0FF66E55
:1000D000000EF7220900F5500EBEF28E12002130FC
:1000E0003033302C2530344C582C2530344C582C9F
:1000F000253032582C253032582C253032582C25BA
:100100003032580D0A00F2CF0EF0F29EF76A200F3F
:10011000F66E010EF7220900F5500EBEF28E1200A7
:1001200021303032302C2530394C550D0A00F2CFB9
:100130000EF0F29EF76A480FF66E010EF7220900E4
:10014000F5500EBEF28E1200482D4272696467654A
:1001500020647269766572207465737420666978AC
:10016000747572650D0A0000F2CF0EF0F29EF76A08
:10017000820FF66E010EF7220900F5500EBEF28EC8
:10018000120048573A303139312046573A30313928
:10019000342E30302E30300D0A0D0A00F2CF0EF022
:1001A000F29EF76AB60FF66E010EF7220900F550BF
:1001B0000EBEF28E120024303031306E6E6E6E5BE9
:1001C00063725D202020202020202020202020205D
:1001D0002020202020202020537461727420746518
:1001E00073742C2072756E206E6E6E6E2063796350
:1001F0006C65732028486578290D0A00F2CF0EF04F
:10020000F29EF76A160FF66E020EF7220900F550FD
:100210000EBEF28E12002130303130615B63725DB0
:1002200020202020202020202020202020202020CE
:1002300020202020202020202830303030207275CF
:100240006E7320636F6E74696E756F75736C792948
:100250000D0A0D0A0000F2CF0EF0F29EF76A700F41
:10026000F66E020EF7220900F5500EBEF28E120055
:1002700024303032305B63725D202020202020202B
:10028000202020202020202020202020202020206E
:1002900020205265706F7274206379636C652063EF
:1002A0006F756E740D0A0000F2CF0EF0F29EF76AC1
:1002B000C20FF66E020EF7220900F5500EBEF28E46
:1002C000120021303032302C6E6E6E6E6E6E6E6E9D
:1002D0006E5B63725D2020202020202020202020C3
:1002E000202020204379636C6520636F756E742035
:1002F00028446563696D616C290D0A0D0A00F2CF0F
:100300000EF0F29EF76A180FF66E030EF722090040
:10031000F5500EBEF28E120024303032315B637223
:100320005D20202020202020202020202020202090
:1003300020202020202020202020436C6561722076
:100340006379636C6520636F756E740D0A00F2CF7C
:100350000EF0F29EF76A680FF66E030EF7220900A0
:10036000F5500EBEF28E12002130303231615B63E7
:10037000725D0D0A0D0A0000F2CF0EF0F29EF76AD0
:10038000920FF66E030EF7220900F5500EBEF28EA4
:10039000120024303033305B63725D202020202037
:1003A000202020202020202020202020202020204D
:1003B000202020205265706F727420746573742041
:1003C000706172616D657465727320284865782963
:1003D0000D0A0000F2CF0EF0F29EF76AEE0FF66EF5
:1003E000030EF7220900F5500EBEF28E12002130E6
:1003F0003033302C747474742C636363632C6161C8
:100400002C62622C78782C79795B63725D202020D5
:10041000747474743A202053746F70207468726519
:1004200073686F6C640D0A00F2CF0EF0F29EF76AEB
:10043000420FF66E040EF7220900F5500EBEF28E42
:100440001200636363633A202053746F7020636FFC
:10045000756E740D0A00F2CF0EF0F29EF76A700FFF
:10046000F66E040EF7220900F5500EBEF28E120051
:1004700061613A202020205269676874206C6567AA
:10048000206F6E2C20206D530D0A0000F2CF0EF06D
:10049000F29EF76AA60FF66E040EF7220900F550D9
:1004A0000EBEF28E120062623A2020202020202010
:1004B000202020202020206F66662C206D530D0AFE
:1004C0000000F2CF0EF0F29EF76ADC0FF66E040E1B
:1004D000F7220900F5500EBEF28E120078783A200D
:1004E0002020204C656674206C656720206F6E2C80
:1004F00020206D530D0A0000F2CF0EF0F29EF76A35
:10050000120FF66E050EF7220900F5500EBEF28EA0
:10051000120079793A20202020202020202020203D
:100520002020206F66662C206D530D0A0D0A0000F6
:10053000F2CF0EF0F29EF76A4A0FF66E050EF72222
:100540000900F5500EBEF28E1200243030333174A3
:100550007474746363636361616262787879795BF0
:1005600063725D20202020202020202053657420ED
:100570007465737420706172616D65746572732047
:1005800028486578290D0A00F2CF0EF0F29EF76A2E
:10059000A20FF66E050EF7220900F5500EBEF28E80
:1005A00012002130303331615B63725D20202020E6
:1005B000202020202020202020202020202020203B
:1005C00020202020747474743A202053746F70209B
:1005D0007468726573686F6C640D0A00F2CF0EF078
:1005E000F29EF76AF60FF66E050EF7220900F55037
:1005F0000EBEF28E120021303034306363636363C9
:10060000636161617878785B63725D2020202020CF
:1006100020202020202020204379636C65207465F1
:1006200073742073746174732028486578290D0AE7
:100630000000F2CF0EF0F29EF76A4C0FF66E060E37
:10064000F7220900F5500EBEF28E12006363636359
:100650006363204379636C6520636F756E740D0A64
:100660000000F2CF0EF0F29EF76A7C0FF66E060ED7
:10067000F7220900F5500EBEF28E12006161612072
:100680002020204C656720612D62206375727265A1
:100690006E740D0A0000F2CF0EF0F29EF76AB00FF2
:1006A000F66E060EF7220900F5500EBEF28E12000D
:1006B000787878202020204C656720782D79206379
:1006C000757272656E740D0A0D0A0000F2CF0EF09D
:1006D000F29EF76AE60FF66E060EF7220900F55055
:1006E0000EBEF28E120020205468652027526967E2
:1006F0006874206C656727206379636C6520697373
:1007000020746865206C656674206869676820617C
:100710006E6420746865207269676874206C6F77F6
:100720002C20692E652E204144430D0A0000F2CF93
:100730000EF0F29EF76A480FF66E070EF7220900D8
:10074000F5500EBEF28E12006D6561737572696EA2
:10075000672063757272656E7420617420746865B9
:100760002072696768742073696465206F662074FD
:1007700068652062726964676520746F2067726FB4
:10078000756E6420616E642074686520274C656610
:10079000740D0A00F2CF0EF0F29EF76AAE0FF66EFD
:1007A000070EF7220900F5500EBEF28E12006C659E
:1007B0006727206379636C6520697320636F6E76A9
:1007C000657273656C7920746865207269676874F6
:1007D000206869676820616E6420746865206C65B4
:1007E0006674206C6F773A2020466F7220746865BB
:1007F000204442392D4D2C0D0A00F2CF0EF0F29E0E
:10080000F76A140FF66E080EF7220900F5500EBEB7
:10081000F28E1200746869732069732070696E73B8
:1008200020322D2F372B20616E6420322B2F372D55
:1008300020726573706563746976656C792E20200B
:100840004C65672063757272656E742063616E20FB
:1008500062652063616C63756C617465640D0A0088
:10086000F2CF0EF0F29EF76A7A0FF66E080EF722BC
:100870000900F5500EBEF28E120066726F6D3A20BE
:10088000496F7574203D2028284144432F31303270
:1008900033292A322E35292F526C6F772E0D0A0DEF
:1008A0000A00F2CF0EF0F29EF76ABC0FF66E080E49
:1008B000F7220900F5500EBEF28E12002020546877
:1008C000652073746F70207468726573686F6C64F0
:1008D0002069732074686520414443207265616417
:1008E000696E6720636F6E736964657265642074F6
:1008F0006F20626520616E206F70656E2062726984
:100900006467650D0A00F2CF0EF0F29EF76A200FC1
:10091000F66E090EF7220900F5500EBEF28E120097
:10092000616E64207468652073746F7020636F75E6
:100930006E7420697320746865206E756D626572CF
:10094000206F662074696D657320284E6F6E2D636D
:100950006F6E7365637574697665292074686520A8
:100960004144430D0A00F2CF0EF0F29EF76A800F69
:10097000F66E090EF7220900F5500EBEF28E120037
:1009800072656164696E672066616C6C7320626574
:100990006C6F772074686174207468726573686F17
:1009A0006C6420616674657220776869636820747E
:1009B00068652074657374206973207465726D694D
:1009C0006E617465642E0D0A0000F2CF0EF0F29E87
:1009D000F76AE40FF66E090EF7220900F5500EBE15
:1009E000F28E12005468652073746F702074687200
:1009F0006573686F6C642063616E2072616E6765F9
:100A00002066726F6D203020746F2039393939209B
:100A1000283130323320746F2039393939206973E5
:100A20002053544F50212920616E640D0A00F2CFEB
:100A30000EF0F29EF76A480FF66E0A0EF7220900D2
:100A4000F5500EBEF28E12007468652073746F70DC
:100A500020636F756E742063616E2072616E6765CE
:100A60002066726F6D203120746F20393939392E2C
:100A70000D0A0D0A0000F2CF0EF0F29EF76A900FF9
:100A8000F66E0A0EF7220900F5500EBEF28E120025
:100A9000202054686520746573742074696D6573D3
:100AA0002061726520696E206D532C206275742060
:100AB0006172652061637475616C6C7920312E30D0
:100AC00032346D532062656361757365206F6620F3
:100AD000746865207761790D0A00F2CF0EF0F29EFE
:100AE000F76AF40FF66E0A0EF7220900F5500EBEF3
:100AF000F28E120074696D6520697320636F756EE4
:100B000074656420696E20746865205049432E2006
:100B100020412073657474696E67206F66202731E9
:100B200030272077696C6C20726573756C7420694E
:100B30006E20616E642061637475616C0D0A000043
:100B4000F2CF0EF0F29EF76A5A0FF66E0B0EF722F6
:100B50000900F5500EBEF28E120074696D65206FAB
:100B6000662031302E32346D532E20204D696E694F
:100B70006D756D206F6E2074696D6520697320310D
:100B80006D532C206D696E696D756D206F666620E2
:100B900074696D6520697320306D532E20204E6F6F
:100BA00074650D0A0000F2CF0EF0F29EF76AC00FD6
:100BB000F66E0B0EF7220900F5500EBEF28E1200F3
:100BC0007468617420356D532069732074686520E2
:100BD0006D696E696D756D20696E7465677261749B
:100BE000696F6E2074696D65207768657265206332
:100BF000757272656E74206973207265616420611C
:100C0000742074686520656E640D0A00F2CF0EF0E2
:100C1000F29EF76A260FF66E0C0EF7220900F550C9
:100C20000EBEF28E12006F6620746865206F6E2013
:100C30006379636C6520616E642073686F7274659C
:100C4000722074696D65732077696C6C20726573AE
:100C5000756C7420696E20696E616363757261746E
:100C600065204144432072656164696E67732E0D8F
:100C70000A00F2CF0EF0F29EF76A8C0FF66E0C0EA1
:100C8000F7220900F5500EBEF28E12004661737411
:100C9000657220696E746567726174696F6E206336
:100CA000616E2062652061636865697665642062B3
:100CB00079207265647563696E6720746865207653
:100CC000616C7565206F6620523920616E64205218
:100CD00031302E0D0A00F2CF0EF0F29EF76AF00FBF
:100CE000F66E0C0EF7220900F5500EBEF28E1200C1
:100CF000546865206D6178696D756D206F6E206137
:100D00006E64206F66662074696D6573206172651C
:100D10002039396D532E0D0A0D0A0000F2CF0EF066
:100D2000F29EF76A360FF66E0D0EF7220900F550A7
:100D30000EBEF28E12002020546865206C65667429
:100D400020627574746F6E2028466163696E672037
:100D5000746865207465737420636F6E6E65637468
:100D60006F7229207374617274732074657374696F
:100D70006E67207768656E20707265737365640DA9
:100D80000A00F2CF0EF0F29EF76A9C0FF66E0D0E7F
:100D9000F7220900F5500EBEF28E1200666F722027
:100DA00032206F72206D6F7265207365636F6E64A1
:100DB000732E2020546865207269676874206275FC
:100DC00074746F6E2073746F707320612074657318
:100DD0007420696E2070726F677265737320696D1D
:100DE0006D6564696174656C790D0A00F2CF0EF06F
:100DF000F29EF76A060FF66E0E0EF7220900F55006
:100E00000EBEF28E1200616E64207768656E2069F6
:100E1000646C6520636C656172732074686520740E
:100E200065737420636F756E7420616674657220DB
:100E300035207365636F6E64732E20205072657366
:100E400073696E6720626F746820627574746F6E68
:100E5000730D0A00F2CF0EF0F29EF76A6E0FF66E77
:100E60000E0EF7220900F5500EBEF28E12006469D4
:100E700073706C617973207468652074696D696E34
:100E80006720706172616D657465727320666F7240
:100E90002035207365636F6E647320616E64207407
:100EA00068656E20646973706C617973207468651D
:100EB000207468726573686F6C640D0A0000F2CF6D
:100EC0000EF0F29EF76AD80FF66E0E0EF7220900AA
:100ED000F5500EBEF28E1200616E6420636F756E67
:100EE00074206C696D69747320756E74696C20650B
:100EF000697468657220627574746F6E20697320FE
:100F000072656C65617365642E0D0A0D0A00F2CF7F
:100F10000EF0F29EF76A280FF66E0F0EF722090008
:100F2000F5500EBEF28E12002020447572696E6775
:100F30002074657374696E672C2064617461206924
:100F400073207472616E736D697474656420746F5C
:100F500020525332333220616E6420646973706CA6
:100F60006179656420696E204845582028746F2097
:100F7000736176650D0A0000F2CF0EF0F29EF76AFB
:100F8000920FF66E0F0EF7220900F5500EBEF28E8C
:100F9000120074696D65292062757420616674653C
:100FA000722074657374696E67206861732073744E
:100FB0006F7070656420616E6420647572696E671D
:100FC00020706172616D6574657220646973706C04
:100FD00061792C2076616C756573206172650D0AEC
:100FE0000000F2CF0EF0F29EF76AFC0FF66E0F0EC5
:100FF000F7220900F5500EBEF28E120073686F776B
:101000006E20696E20646563696D616C2E202041DD
:101010006E7920525332333220636F6D6D616E648E
:1010200020726563656976656420647572696E67B0
:101030002074657374696E672077696C6C207374B3
:101040006F70207468650D0A0000F2CF0EF0F29EFA
:10105000F76A640FF66E100EF7220900F5500EBE07
:10106000F28E120074657374696E6720696D6D6528
:1010700064696174656C792E0D0A0D0A0000F2CF67
:101080000EF0F29EF76A980FF66E100EF722090026
:10109000F5500EBEF28E120044535542392D4D20AC
:1010A000636F6E6E6563746F722070696E206F750A
:1010B000743A0D0A0000F2CF0EF0F29EF76AD00FDC
:1010C000F66E100EF7220900F5500EBEF28E1200D9
:1010D0003120202052696768742D6C65672048694B
:1010E0006768202020205768656E206E6F7420741A
:1010F000657374696E672C20706F7473206D6179ED
:10110000206265207265616420617420482D746FCF
:101110002D4D20616E64204D2D746F2D4C0D0A00F5
:10112000F2CF0EF0F29EF76A3A0FF66E110EF7222A
:101130000900F5500EBEF28E1200322020205269B6
:101140006768742D6C6567204D6964646C65202048
:10115000666F722074686520707572706F73652099
:101160006F662073657474696E67207468652062A9
:1011700072696467652063757272656E742E2020D3
:101180004A7573742062650D0A00F2CF0EF0F29E6C
:10119000F76AA40FF66E110EF7220900F5500EBE85
:1011A000F28E12003320202052696768742D6C651E
:1011B00067204C6F77202020202073757265207483
:1011C0006F2072656D6F766520616E79205555547C
:1011D000207768656E2073657474696E6720746823
:1011E0006520706F74732E0D0A00F2CF0EF0F29E20
:1011F000F76A040FF66E120EF7220900F5500EBEC4
:10120000F28E1200202020202D2D2D2D2D2D2D2D64
:101210002D2D2D2D2D2D2D2D0D0A0000F2CF0EF090
:10122000F29EF76A360FF66E120EF7220900F5509D
:101230000EBEF28E1200362020204C6566742D6C96
:1012400065672020486967680D0A0000F2CF0EF03C
:10125000F29EF76A660FF66E120EF7220900F5503D
:101260000EBEF28E1200372020204C6566742D6C65
:10127000656720204D6964646C650D0A0000F2CF3B
:101280000EF0F29EF76A980FF66E120EF722090022
:10129000F5500EBEF28E1200382020204C65667488
:1012A0002D6C656720204C6F770D0A00F2CF0EF091
:1012B000F29EF76AC60FF66E120EF7220900F5507D
:1012C0000EBEF28E12003420202047726F756E64BD
:1012D0000D0A0000F2CF0EF0F29EF76AEE0FF66EE6
:1012E000120EF7220900F5500EBEF28E12003920C0
:1012F00020204C6566742028537461727429206222
:101300007574746F6E2C20616374697665206C6FE0
:10131000772077697468206E6F204553442070727F
:101320006F74656374696F6E0D0A0000F2CF0EF082
:10133000F29EF76A460FF66E130EF7220900F5507B
:101340000EBEF28E1200352020205269676874208C
:101350002853746F702F52657365742920627574F9
:10136000746F6E2C20616374697665206C6F7720D2
:1013700077697468206E6F204553442070726F74D3
:10138000656374696F6E0D0A0D0A0000F2CF0EF0EE
:10139000F29EF76AA60FF66E130EF7220900F550BB
:1013A0000EBEF28E1200436170747572652074680F
:1013B0006973206D656E7520746F2066696C652099
:1013C000696620746865207465726D696E616C2051
:1013D0007363726F6C6C206261636B20627566660A
:1013E0006572206D616B6573206974206861726439
:1013F0000D0A0000F2CF0EF0F29EF76A0E0FF66EA5
:10140000140EF7220900F5500EBEF28E1200746F12
:1014100020726561642074686520746F70206F6647
:1014200020746865206D656E75210D0A0D0A000037
:10143000F2CF0EF0F29EF76A4A0FF66E140EF72204
:101440000900F5500EBEF28E120053797374656D6B
:1014500055700000F2CF0EF0F29EF76A6E0FF66E36
:10146000140EF7220900F5500EBEF28E12005468D9
:10147000723A2530344C5500F2CF0EF0F29EF76AE6
:10148000920FF66E140EF7220900F5500EBEF28E82
:1014900012005374703A2530344C55009EA8FED784
:1014A000AD6E000C9EAAFED7AECF6FF2020119B648
:1014B00075D019B809D06F51240805E11988199A17
:1014C000240E326E316A6AD06F51240A000103E0A3
:1014D000290A06E033D0199A240E326E316A5FD0A1
:1014E000199831522AE033501C5C27E119BA02D016
:1014F000312C04D0198E660E316E1FD019BC05D068
:10150000020E315C1C6E198618D02F50325CD880C8
:101510003054326E010E315C036A1C0FE96E000E0E
:101520000320EA6EEF50325C05E1030E315C1C6E65
:10153000198603D0198E630E316E31D002016F51BE
:10154000322619BA04D0198A6FC22FF027D0199AFF
:101550006FC230F02FC06FF26F3BF00E6F172FACE1
:1015600002D0900E6F2730500F0B6F2730AC02D097
:10157000090E6F27036A31501C0FE96E000E03201D
:10158000EA6E6FC2EFFF312A3150120807E2199854
:1015900033501C5C03E1198E6F0E316E000119A6E9
:1015A00031D01D5007E0010A0EE0030A17E0050ADA
:1015B0001FE028D0198E1C5203E1300E316E02D08C
:1015C000660E316E1FD0198E1C2C05D01EC033F054
:1015D000610E316E02D0660E316E14D0198E1C521F
:1015E00004E1197C610E316E02D0660E316E0AD0B4
:1015F000198E1C5204E13480610E316E02D0660EE9
:10160000316E00D019AE7CD0199E210E47DF33C059
:101610006FF202016F3B6F510F0B300F6F6F6F5105
:10162000390802E2070E6F27210E6F25326E6F51C7
:10163000000134DF33500F0B300F02016F6F6F5119
:10164000390802E2070E6F276F51000127DF020100
:101650006F51322619A624D01996300E00011EDFD4
:10166000300E1D240201706F000118DF300E32248D
:101670001D24300F326E1D5212E11C5210E1300E4B
:101680000DDF310E0BDF390E09DF340E07DF300EB0
:1016900005DF300E03DF300E01DF5E0E3226020161
:1016A00031500001FBDE3150322619AC1DD032C062
:1016B0006FF202016F3B6F510F0B300F6F6F6F5165
:1016C000390802E2070E6F276F510001E7DE325042
:1016D0000F0B300F02016F6F6F51390802E2070ED6
:1016E0006F276F510001DADE0D0ED8DE0A0ED6DE4E
:1016F00034A006D0000ED2DE000ED0DE3490FF0003
:10170000000E9EBA010E0108D8B4CCD69E9A2CEFDA
:1017100000F0200E896E0A0E8A6EC00E8B6E1F0EB0
:10172000926E936A840E946EC150C00B1D09C16EF7
:10173000C050C00B3F09C06EC08EC280C69A010E59
:10174000C66E000EC76ED190C10ED56ECD6A000E6A
:10175000CA6E000ECB6E070EB46E9250926E0400ED
:10176000200E006E002EFED700D0B450A19CB56AAA
:101770009D8AC00EF2123492396A386A376A366A24
:10178000F2CF52F2F29EA96AA69CA69EA680A8500D
:10179000020152BFF28E536FF2CF54F2F29E010E4D
:1017A000A96EA69CA69EA680A85054BFF28E556F27
:1017B00053C23BF055C23AF03B50260809E2FF0AFB
:1017C00003E13A500F0804E2270E3B6E0F0E3A6E0B
:1017D000F2CF52F2F29E020EA96EA69CA69EA680A1
:1017E000A85052BFF28E536FF2CF54F2F29E030E06
:1017F000A96EA69CA69EA680A85054BFF28E556FD7
:1018000053C23DF055C23CF03D50260809E2FF0AA4
:1018100003E13C500F0804E2270E3D6E0F0E3C6EB4
:101820003C5205E13D5203E13D6A010E3C6EF2CFB0
:1018300052F2F29E040EA96EA69CA69EA680A85007
:1018400052BFF28E406E4050630802E2630E406E5B
:10185000405202E1010E406EF2CF52F2F29E050EAE
:10186000A96EA69CA69EA680A85052BFF28E416E7D
:101870004150630802E2630E416EF2CF52F2F29ED3
:10188000060EA96EA69CA69EA680A85052BFF28EF8
:10189000426E4250630802E2630E426E425202E11F
:1018A000010E426EF2CF52F2F29E070EA96EA69C76
:1018B000A69EA680A85052BFF28E436E4350630886
:1018C00002E2630E436E3F6A3E6A456A446A476AB3
:1018D000466A0101486B496B02014A6B4B6B000180
:1018E0003BEF18F00201546B545113080AE3036AEA
:1018F00054511C0FE96E000E0320EA6EEF6A542B60
:10190000F3D7316A53C232F052C233F019961998A4
:10191000199A199C199E3490000141EF18F0020E9B
:10192000EA6E640EE96EEF5011E00C0E016EBF0E10
:10193000006E0400002EFDD7012EF9D7F70E006EC1
:10194000002EFED700000400EF2EEFD7000C02019E
:10195000646B8B8200D0000082A401D0648182A6D7
:1019600001D0648382A801D0648582AA01D06487F3
:101970008B9200D0000064C201F00001000C899A33
:10198000949494969498949A020163A9829463B96A
:10199000828463AB829663BB828663AD829863BDAB
:1019A000828863AF829A63BF828A0001D0DF352CC0
:1019B00005D00A0E0201646F0001B1DF020163A1CC
:1019C000829463B1828463A3829663B3828663A5A3
:1019D000829863B5828863A7829A63B7828A00017E
:1019E000B6DF352C05D00A0E0201646F000197DFC7
:1019F000000C010E356E929A949094928B92000096
:101A00008B900000899A320E0201646F000187DF1B
:101A1000330E0201636F0001B2DF320E0201636F09
:101A20000001ADDF280E0201636F0001A8DF060E82
:101A30000201636F0001A3DF0C0E0201636F00015E
:101A40009EDF010E0201636F000199DF46EF18F07F
:101A5000898A948494869488948A79DF0138020173
:101A6000636FF00E6317000172DF01500201631310
:101A700063C201F00001000C8B90EADF01C063F249
:101A8000020101AE02D00001F8D70001000C356A56
:101A9000F3DF8B8062C263F272DF000C356AECDF29
:101AA0008B905EC263F26BDF000C006A016A026A0F
:101AB000036A02016A6B6B6B6C6B6D6B6951681129
:101AC000671166112CE0200E6E6FD8906237633775
:101AD000643765376A376B376C376D3769516D5DC1
:101AE00008E168516C5D05E167516B5D02E166518B
:101AF0006A5D0FE366516A5F6751D8A0673D6B5F0F
:101B00006851D8A0683D6C5F6951D8A0693D6D5F90
:101B1000D88000360136023603366E2FD6D7020E35
:101B2000EA6E6A0EE96E0001000CE95002015A6F7C
:101B30003B0E616F9A0E606FCA0E5F6F5E6B0A0E8E
:101B40005C6F59C265F258C264F257C263F256C262
:101B500062F261C269F260C268F25FC267F25EC29D
:101B600066F20001A2DF0150EFCF56F2ECCF57F240
:101B7000ECCF58F2ECCF59F2005213E102015C5164
:101B8000010AD8A402D000010CD05A510CE00F0B6E
:101B90005C5D01E00FE25ABF0DD05ABD04D0200EAB
:101BA00003D002015A6B300E002600C062F2000121
:101BB0006EDF020161C265F260C264F25FC263F26D
:101BC0005EC262F2696B686B676B0A0E666F00013A
:101BD0006CDF03C061F202C060F201C05FF200C0BE
:101BE0005EF202015C2FADD7000167EF0EF0EACF85
:101BF0005EF2E9CF5DF202015739F009596F5927BA
:101C0000E20F5A6F320F5C6F57510F0B5A275A274A
:101C10005C27E90F5B6F5B275B2756390F0B5B2750
:101C20005C275B375C375C1F5C3756510F0B5C27BA
:101C30005937070E586F0A0E5B075C27FDE35A07FA
:101C40005B27FDE359075A27FDE358075927FDE3B2
:101C5000020EEA6E580EE96E070E5D155D9DE926CF
:101C60005C0EE95CD8B45D8DEF50006E08E15DBD9F
:101C700006D05DB915D05DB702D0200E03D05D87C8
:101C80005D99300E0026EACF57F2E9CF56F200C038
:101C900062F20001FCDE57C2EAFF56C2E9FF020110
:101CA000EE505DADDDD70001000C34A42DD0800EC8
:101CB00002015E6F0001F2DE480EE96E39C059F292
:101CC00038C058F237C057F236C056F22ED7C00E81
:101CD00002015E6F0001E2DE610E0201626F00012F
:101CE000D6DE0A0EE96E45C057F244C056F27FDFD9
:101CF000780E0201626F0001CADE0A0EE96E47C06B
:101D000057F246C056F273DF000C456A446A476AD0
:101D1000466A396A386A376A366AC7DF000C1A2A97
:101D2000D8B41B2A1A3C0CD01B507F0809E119803B
:101D300019728A9819B28A8819841B6A1A6A01D0A2
:101D400019906AEF18F0020157BF10D00F0E006E05
:101D5000563900160A0E005C03E2300E002602D04F
:101D60005751002600509EA8FED7AD6E0F0E561795
:101D70000A0E565D02E2300E02D0579F5751562789
:101D800056519EA8FED7AD6E0001000CE95002012D
:101D90005A6F3B0E616F9A0E606FCA0E5F6F5E6B7B
:101DA0000A0E5C6F59C265F258C264F257C263F200
:101DB00056C262F261C269F260C268F25FC267F243
:101DC0005EC266F2000171DE0150EFCF56F2ECCF39
:101DD00057F2ECCF58F2ECCF59F2005213E1020166
:101DE0005C51010AD8A402D000010CD05A510CE079
:101DF0000F0B5C5D01E00EE25ABF0CD05ABD04D05F
:101E0000200E03D002015A6B300E002600509EA80F
:101E1000FED7AD6E61C265F260C264F25FC263F26A
:101E20005EC262F2696B686B676B0A0E666F0001D7
:101E30003CDE03C061F202C060F201C05FF200C08C
:101E40005EF202015C2FAED70001FBEF10F0020141
:101E50005651F00B5A6F5A3B300E5A275A513908D7
:101E600002E2070E5A2758C2E9FF59C2EAFF5AC2D6
:101E7000EFFF56510F0B5B6F5C6B300E5B255A6F9B
:101E80005A51390802E2070E5A27010E5825E96E09
:101E9000000E5921EA6E5AC2EFFF0001000CABA2FE
:101EA00002D0AB98AB8819A66EEF15F01D50300A22
:101EB00011E0010AD8B471D0110AD8B47FD1010A57
:101EC000D8B4A5D1310AD8B4ACD1EF0AD8B4B7D1BF
:101ED0003CEF15F01C525DE10201566B56510001BA
:101EE00062EC00F00201562B00014EEC0AF0060EE7
:101EF0000201565DF3E13BC056F2370E576F000109
:101F000022DF3AC056F2370E0201576F00011BDF85
:101F10002C0E4EEC0AF03DC056F2370E0201576F00
:101F2000000111DF3CC056F2370E0201576F00016D
:101F30000ADF2C0E4EEC0AF040C056F2370E0201BA
:101F4000576F000100DF2C0E4EEC0AF041C056F234
:101F5000370E0201576F0001F6DE2C0E4EEC0AF030
:101F600042C056F2370E0201576F0001ECDE2C0E14
:101F70004EEC0AF043C056F2370E0201576F0001D3
:101F8000E2DE0D0E4EEC0AF00A0E4EEC0AF01C6A70
:101F900002D0660E1C6E3FEF15F01C500808D8A446
:101FA00008D1F29CF29EF2BEFDD71EC053F21FC0B4
:101FB00052F20201535126080DE2FF0A03E1525189
:101FC0000F0808E2270E536F0F0E526F53C21EF018
:101FD00052C21FF053C23BF052C23AF020C053F23B
:101FE00021C052F2535126080DE2FF0A03E152517B
:101FF0000F0808E2270E536F0F0E526F53C21EF0E8
:1020000052C21FF0525307E1535305E1536B010EC7
:10201000526F206A216E53C23DF052C23CF02252F0
:1020200002E1010E226E2250630802E2630E226E6C
:1020300022C040F02350630802E2630E236E23C0E7
:1020400041F0245202E1010E246E2450630802E2A2
:10205000630E246E24C042F02550630802E2630E32
:10206000256E25C043F0A96A1EC0A8FFA69CA69EA7
:10207000A684F2CF00F0F29E0F01550EA76EAA0EB5
:10208000A76EA682A6B2FED7A6940050F212010E49
:10209000A96E1FC0A8FFA69CA69EA684F2CF00F042
:1020A000F29E550EA76EAA0EA76EA682A6B2FED706
:1020B000A6940050F212020EA96E20C0A8FFA69CA2
:1020C000A69EA684F2CF00F0F29E550EA76EAA0E31
:1020D000A76EA682A6B2FED7A6940050F212030EF7
:1020E000A96E21C0A8FFA69CA69EA684F2CF00F0F0
:1020F000F29E550EA76EAA0EA76EA682A6B2FED7B6
:10210000A6940050F212040EA96E22C0A8FFA69C4D
:10211000A69EA684F2CF00F0F29E550EA76EAA0EE0
:10212000A76EA682A6B2FED7A6940050F212050EA4
:10213000A96E23C0A8FFA69CA69EA684F2CF00F09D
:10214000F29E550EA76EAA0EA76EA682A6B2FED765
:10215000A6940050F212060EA96E24C0A8FFA69CF9
:10216000A69EA684F2CF00F0F29E550EA76EAA0E90
:10217000A76EA682A6B2FED7A6940050F212070E52
:10218000A96E25C0A8FFA69CA69EA684F2CF00F04B
:10219000F29E550EA76EAA0EA76EA682A6B2FED715
:1021A000A6940050F212C00EF212610E1C6E03D003
:1021B0000001660E1C6E00013FEF15F01C5223E17A
:1021C0000201566B5651000183EC00F00201562BC0
:1021D00000014EEC0AF0060E0201565DF3E1490ED5
:1021E000E96E39C059F238C058F237C057F236C0DC
:1021F00056F20001CBD50D0E4EEC0AF00A0E4EEC55
:102200000AF01C6A02D0660E1C6E3FEF15F01C52DD
:1022100004E1610E1C6E79DD02D0660E1C6E3FEF8C
:1022200015F01C50020807E11EC03FF01FC03EF031
:1022300034821C6A02D0660E1C6E3FEF15F01C52F1
:10224000D8A438EF15F00201566B5651000197ECF7
:1022500000F00201562B00014EEC0AF01E0E0201A6
:10226000565DF3E1566B56510001B4EC00F00201EB
:10227000562B00014EEC0AF0190E0201565DF3E1F7
:10228000566B56510001CEEC00F00201562B0001B6
:102290004EEC0AF0450E0201565DF3E1566B5651C5
:1022A0000001FEEC00F00201562B00014EEC0AF09A
:1022B0003E0E0201565DF3E1566B565100012BECC8
:1022C00001F00201562B00014EEC0AF0360E02011D
:1022D000565DF3E1566B5651000154EC01F00201DA
:1022E000562B00014EEC0AF03B0E0201565DF3E165
:1022F000566B565100017FEC01F00201562B000194
:102300004EEC0AF0350E0201565DF3E1566B565164
:102310000001A7EC01F00201562B00014EEC0AF07F
:102320000E0E0201565DF3E1566B56510001BCECF6
:1023300001F00201562B00014EEC0AF0400E0201A2
:10234000565DF3E1566B56510001EAEC01F00201D3
:10235000562B00014EEC0AF0390E0201565DF3E1F6
:10236000220E566F200E00014EEC0AF00201562F8D
:10237000F9D7566B5651000114EC02F00201562BAE
:1023800000014EEC0AF0130E0201565DF3E1220E3D
:10239000566F200E00014EEC0AF00201562FF9D7BD
:1023A000566B565100012BEC02F00201562B000136
:1023B0004EEC0AF01A0E0201565DF3E1220E566F42
:1023C000200E00014EEC0AF00201562FF9D7566B91
:1023D0005651000146EC02F00201562B00014EEC72
:1023E0000AF01A0E0201565DF3E1220E566F200E1E
:1023F00000014EEC0AF00201562FF9D7566B5651E8
:10240000000161EC02F00201562B00014EEC0AF0D3
:102410001A0E0201565DF3E1220E566F200E0001E6
:102420004EEC0AF00201562FF9D7566B56510001B7
:102430007CEC02F00201562B00014EEC0AF01C0E5F
:102440000201565DF3E1566B5651000198EC02F023
:102450000201562B00014EEC0AF03D0E0201565DC2
:10246000F3E1566B56510001C4EC02F00201562B09
:1024700000014EEC0AF0390E0201565DF3E1220E26
:10248000566F200E00014EEC0AF00201562FF9D7CC
:10249000566B5651000114EC02F00201562B00015C
:1024A0004EEC0AF0130E0201565DF3E1220E566F58
:1024B000200E00014EEC0AF00201562FF9D7566BA0
:1024C000565100012BEC02F00201562B00014EEC9C
:1024D0000AF01A0E0201565DF3E1220E566F200E2D
:1024E00000014EEC0AF00201562FF9D7566B5651F7
:1024F000000146EC02F00201562B00014EEC0AF0FE
:102500001A0E0201565DF3E1220E566F200E0001F5
:102510004EEC0AF00201562FF9D7566B56510001C6
:1025200061EC02F00201562B00014EEC0AF01A0E8B
:102530000201565DF3E1220E566F200E00014EECB3
:102540000AF00201562FF9D7566B565100017CEC68
:1025500002F00201562B00014EEC0AF01C0E0201A3
:10256000565DF3E1566B56510001EEEC02F00201AC
:10257000562B00014EEC0AF03A0E0201565DF3E1D3
:10258000220E566F200E00014EEC0AF00201562F6B
:10259000F9D7566B5651000119EC03F00201562B86
:1025A00000014EEC0AF0140E0201565DF3E1220E1A
:1025B000566F200E00014EEC0AF00201562FF9D79B
:1025C000566B5651000131EC03F00201562B00010D
:1025D0004EEC0AF0180E0201565DF3E1220E566F22
:1025E000200E00014EEC0AF00201562FF9D7566B6F
:1025F000565100014BEC03F00201562B00014EEC4A
:102600000AF01A0E0201565DF3E1566B56510001B5
:1026100066EC03F00201562B00014EEC0AF0460E68
:102620000201565DF3E1566B5651000197EC03F041
:102630000201562B00014EEC0AF04B0E0201565DD2
:10264000F3E1566B56510001CAEC03F00201562B20
:1026500000014EEC0AF04B0E0201565DF3E1566BA1
:1026600056510001FDEC03F00201562B00014EEC27
:102670000AF04B0E0201565DF3E1566B5651000114
:1026800030EC04F00201562B00014EEC0AF0270E4C
:102690000201565DF3E1566B5651000151EC04F016
:1026A0000201562B00014EEC0AF0490E0201565D64
:1026B000F3E1566B5651000183EC04F00201562BF6
:1026C00000014EEC0AF0450E0201565DF3E1566B37
:1026D00056510001B3EC04F00201562B00014EEC00
:1026E0000AF0480E0201565DF3E1566B56510001A7
:1026F000E5EC04F00201562B00014EEC0AF0490E05
:102700000201565DF3E1566B5651000117EC05F0DE
:102710000201562B00014EEC0AF02C0E0201565D10
:10272000F3E1566B565100013BEC05F00201562BCC
:1027300000014EEC0AF0490E0201565DF3E1566BC2
:10274000565100016DEC05F00201562B00014EECD4
:102750000AF04A0E0201565DF3E1566B5651000134
:10276000A0EC05F00201562B00014EEC0AF04A0ED7
:102770000201565DF3E1566B56510001D3EC05F0B2
:102780000201562B00014EEC0AF04B0E0201565D81
:10279000F3E1566B5651000106EC06F00201562B90
:1027A00000014EEC0AF04B0E0201565DF3E1566B50
:1027B0005651000139EC06F00201562B00014EEC97
:1027C0000AF0490E0201565DF3E1566B56510001C5
:1027D0006BEC06F00201562B00014EEC0AF02A0EBB
:1027E0000201565DF3E1566B565100018EEC06F086
:1027F0000201562B00014EEC0AF04B0E0201565D11
:10280000F3E1566B56510001C1EC06F00201562B64
:1028100000014EEC0AF04F0E0201565DF3E1566BDB
:1028200056510001F6EC06F00201562B00014EEC69
:102830000AF04D0E0201565DF3E1566B5651000150
:102840002AEC07F00201562B00014EEC0AF04E0E66
:102850000201565DF3E1566B565100015FEC07F043
:102860000201562B00014EEC0AF0350E0201565DB6
:10287000F3E1566B5651000187EC07F00201562B2D
:1028800000014EEC0AF04E0E0201565DF3E1566B6C
:1028900056510001BCEC07F00201562B00014EEC32
:1028A0000AF04E0E0201565DF3E1566B56510001DF
:1028B000F1EC07F00201562B00014EEC0AF04C0E31
:1028C0000201565DF3E1566B5651000125EC08F00C
:1028D0000201562B00014EEC0AF0180E0201565D63
:1028E000F3E1566B565100013FEC08F00201562B04
:1028F00000014EEC0AF01C0E0201565DF3E1566B2E
:10290000565100015BEC08F00201562B00014EEC21
:102910000AF04F0E0201565DF3E1566B565100016D
:1029200090EC08F00201562B00014EEC0AF04F0E1D
:102930000201565DF3E1566B56510001C5EC08F0FB
:102940000201562B00014EEC0AF0450E0201565DC5
:10295000F3E1566B56510001F5EC08F00201562BDD
:1029600000014EEC0AF0160E0201565DF3E1566BC3
:10297000565100010EEC09F00201562B00014EECFD
:102980000AF0140E0201565DF3E1566B5651000138
:1029900026EC09F00201562B00014EEC0AF0160E4F
:1029A0000201565DF3E1566B565100013FEC09F010
:1029B0000201562B00014EEC0AF0130E0201565D87
:1029C000F3E1566B56510001F5EC08F00201562B6D
:1029D00000014EEC0AF0160E0201565DF3E1566B53
:1029E0005651000156EC09F00201562B00014EEC45
:1029F0000AF00C0E0201565DF3E1566B56510001D0
:102A00006AEC09F00201562B00014EEC0AF03C0E74
:102A10000201565DF3E1566B5651000196EC09F048
:102A20000201562B00014EEC0AF0440E0201565DE5
:102A3000F3E1566B56510001C6EC09F00201562B2A
:102A400000014EEC0AF04C0E0201565DF3E1566BAC
:102A500056510001FAEC09F00201562B00014EEC30
:102A60000AF0200E0201565DF3E11C6A03D000015A
:102A7000660E1C6E000103D03F0E1C6E00D01C526F
:102A80002CE0210E4EEC0AF00201576B33C056F2D7
:102A9000596B2F0E586F000127EC0FF02F504EECA2
:102AA0000AF030504EEC0AF00201576B1DC056F28E
:102AB000596B2F0E586F000127EC0FF02F504EEC82
:102AC0000AF030504EEC0AF01C504EEC0AF00D0E9D
:102AD0004EEC0AF00A0E4EEC0AF019966CEF18F064
:102AE0008B9028EC0DF001C05EF2000E020101BED9
:102AF000010E016E000190EF15F00400ACA20FD0A2
:102B000001014951485D0AE0036A4851480FE96EE6
:102B1000000E0320EA6EEFCFADFF482B0001E0D797
:102B200001521DE102014B514A5D18E0036A4A510E
:102B30004A0FE96E010E0320EA6EEFCF5DF25DAF42
:102B400006D05DC25EF200014EEC0DF005D05DC214
:102B500062F2000147EC0DF002014A2B0001F2A4E1
:102B600005D0F294010E016E04D003D0000E016E68
:102B700000D0000C8A50F00B02015D6F5D510A0914
:102B80008A6E0400200E006E002EFED700D00001D9
:102B9000000CF0DF8A808A923CEF16F0036A020193
:102BA0004B514A0FE96E010E0320EA6E5FC2EFFF40
:102BB0004B2B0001000C02015EBF11D00F0E006E06
:102BC0005D3900160A0E005C03E2300E002602D0CA
:102BD0005E51002600C05FF20001E0DF02010F0E2F
:102BE0005D170A0E5D5D02E2300E02D05E9F5E51FF
:102BF0005D275DC25FF20001D1DF000C036A0101B5
:102C00004951480FE96E000E0320EA6E5FC2EFFFE4
:102C1000492B0001000C02015EBF11D00F0E006EA7
:102C20005D3900160A0E005C03E2300E002602D069
:102C30005E51002600C05FF20001E0DF02010F0ECE
:102C40005D170A0E5D5D02E2300E02D05E9F5E519E
:102C50005D275DC25FF20001D1DF000C8BDF8A844B
:102C60008A96BFEF16F0010E3626D8B0372AD8B4B0
:102C7000382AD8B4392A8DD7000E016EC250C30B42
:102C80000110C26E40500A0DF3500201586B576F8D
:102C9000575302E158530BE000012FDF015205E0CA
:102CA00002015751D8B4580757070201F1D7C28221
:102CB000C2B2FED7C3CF59F2C4CF5AF234A421D046
:102CC000800E5F6F00016ADF39C05DF2370E0201CE
:102CD0005E6F000170DF38C05DF2370E02015E6F7B
:102CE000000169DF37C05DF2370E02015E6F00013F
:102CF00062DF36C05DF2370E02015E6F00015BDFFE
:102D000002015D6B5D5100014FEC00F002015D2B93
:102D1000006E5F6F000172DF060E02015D5DF2E181
:102D200038C05DF2370E5E6F000175DF37C05DF2AF
:102D3000370E02015E6F00016EDF36C05DF2370EA6
:102D400002015E6F000167DF15DF415216E041505E
:102D50000A0DF3500201586B576F575302E1585355
:102D60000BE00001CADE015205E002015751D8B460
:102D7000580757070201F1D70001FCDE6FD7040E98
:102D8000016EC250C30B0110C26E42500A0DF350C7
:102D90000201586B576F575302E158530BE0000183
:102DA000ACDE015205E002015751D8B4580757076D
:102DB0000201F1D7C282C2B2FED7C3CF5BF2C4CF49
:102DC0005CF234A42BD0C00E5F6F0001E7DE610E11
:102DD00002015F6F0001E2DE5AC25DF2B70E02012E
:102DE0005E6F0001E8DE59C25DF2370E02015E6FD0
:102DF0000001E1DE780E02015F6F0001CFDE5CC2F0
:102E00005DF2B70E02015E6F0001D5DE5BC25DF2BE
:102E1000370E02015E6F0001CEDE02012C0E5F6FE5
:102E20000001ECDE5AC25DF2B70E02015E6F0001D6
:102E3000F2DE59C25DF2370E02015E6F0001EBDE79
:102E40002C0E02015F6F0001D9DE5CC25DF2B70E8D
:102E500002015E6F0001DFDE5BC25DF2370E020130
:102E60005E6F0001D8DE0D0E02015F6F0001C6DE4D
:102E70000A0E02015F6F0001C1DE7CDE435216E0E4
:102E800043500A0DF3500201586B576F575302E13C
:102E900058530BE0000131DE015205E002015751A9
:102EA000D8B4580757070201F1D7000163DE5AC2B0
:102EB00045F059C244F05CC247F05BC246F00201E3
:102EC0005A513B5C04E30AE159513A5C07E25C5118
:102ED0003B5C08E303E15B513A5C04E3010E016EE5
:102EE00004D003D0000E016E00D00001000C0201DE
:102EF000556B566B3E521EE13F521CE119B619D07C
:102F000004000001B0DE0201549101B0548154A1CB
:102F100003D0552BD8B4562B19B609D03D50565D69
:102F200004E305E13C50555D02E280B401D001D0DC
:102F3000E5D725D03FC053F23EC052F2525302E1D2
:102F400053531DE0040000018EDE0201549101B0D4
:102F5000548154A103D0552BD8B4562B19B609D09F
:102F60003D50565D04E305E13C50555D02E280B4FE
:102F700001D005D05251D8B453075207DFD7000112
:102F800092EF18F002015551016A545D03E254C2F8
:102F900000F00CD0006A080E566F543700365551B9
:102FA000005CD8B0006E0136562FF7D70001000C38
:102FB000015052C254F2640E0201556F0001E2DF6B
:102FC00000C052F20150300E08E1020153A310D0AC
:102FD00053B70ED053B9200E04D002015397539922
:102FE0005381012601C062F2000147EC0DF002019D
:102FF00052C254F20A0E556F0001C4DF00C052F2F3
:103000000150300E08E1020153B70BD053A109D093
:1030100053B9200E0001012601C062F247EC0DF009
:103020000201300E522752C262F2000147EC0DF04D
:10303000000CF86AD09E088EEA6AE96AB886560ED5
:10304000AF6E000EB06EA60EAC6E900EAB6EC150A1
:10305000C00B0F09C16E070EB46E19901992199426
:103060001A6A1B6A02014C6B4D6B4F6B506B516BB4
:10307000000189EF0BF00201526B536B000172EFFC
:103080000CF082A420D03484F9EF0CF00201526BD2
:103090005251000118EC0AF00201522B006E626FCF
:1030A000000147EC0DF0080E0201525DF1E1080E3F
:1030B000526FFA0E646F00018FEC0CF00201522F78
:1030C000F8D702D000013494000185EC0EF0040022
:1030D0008FEF0EF04FEF0FF002014E9100010DDD6A
:1030E000015210E002014C2BD8B44D2B4D51020877
:1030F00008E2FF0A03E14C51D00803E24D6B4C6B30
:103100004E81000134A21ED03492320E0201646F4F
:1031100000018FEC0CF002014D6B4C6B4F6B506B50
:103120000001E5D602014B514A5D05E1010149511B
:10313000485D05E0020104000001DFDCF3D7000177
:1031400055EC0EF002014EA1C9D080B4A8D080B8D1
:10315000A6D051516308D8A0A1D0512B506B4F6B12
:103160005151320858E1800E5E6F00014EEC0DF0B7
:10317000610E0201626F000147EC0DF0200E0201AA
:10318000626F000147EC0DF02B0E0201626F00012F
:1031900047EC0DF040C052F2010E0201536F0001E6
:1031A00007DF2D0E0201626F000147EC0DF041C0F8
:1031B00052F2010E0201536F0001FADEC00E02014D
:1031C0005E6F00014EEC0DF0780E0201626F00019F
:1031D00047EC0DF0200E0201626F000147EC0DF08C
:1031E0002B0E0201626F000147EC0DF042C052F25B
:1031F000010E0201536F0001DBDE2D0E0201626F32
:10320000000147EC0DF043C052F2010E0201536F72
:103210000001CEDE02015151630840E2800E5E6F74
:1032200000014EEC0DF00201526B525100012AECEC
:103230000AF00201522B006E626F000147EC0DF0A4
:10324000040E0201525DF1E1090EE96E3BC057F236
:103250003AC056F20001F7EC0DF0C00E02015E6FAD
:1032600000014EEC0DF00201526B525100013CEC9A
:103270000AF00201522B006E626F000147EC0DF064
:10328000040E0201525DF1E1090EE96E3DC057F2F4
:103290003CC056F20001F7EC0DF002011FD0515175
:1032A000310804E2000155EC0EF00201516B80B4CC
:1032B0000AD04F2B4F51310805E24F6B000185ECCE
:1032C0000EF0020101D04F6B80B807D0502B505147
:1032D000130802E2506B348201D0506B0001F7D624
:0232E0000300E9
:020000040030CA
:0E0000000046060F000181000FC00FE00F4008
:00000001FF
